:0A00360000010202030304040505A3
:100FB200C216C213D215C214120DB81213BA1210ED
:100FC200DE121354750A0F750B0075120F7513128A
:100FD20075080F75091C75100F75114A75140F7578
:100FE200157890E680E030E70E85080C85090D85BE
:100FF200100E85110F800C85100C85110D85080EC1
:1010020085090FD2E843D82090E668E04409F090C1
:10101200E65CE0443DF0D2AF90E680E020E105D20C
:10102200171212CDE58030E2107FF47E01121148D2
:1010320090E680E054F7F080031213F7538EF8C263
:1010420016E58020E2031213F7301405120762C27C
:061052001412040480EBFF
:1013F70090E680E04408F0E58030E2FB7FF47E0170
:0B14070012114890E680E054F7F0223C
:1007620090E6B9E070030208351470030208D6243B
:10077200FE700302096224FB700302082F14700347
:1007820002082914700302081D14700302082324AE
:100792000560030209C990E6BBE024FE602C1460E8
:1007A2004724FD601614603124067065E50A90E660
:1007B200B3F0E50B90E6B4F00209D5E51290E6B38A
:1007C200F0E51390E6B4F00209D5E50C90E6B3F03B
:1007D200E50D90E6B4F00209D5E50E90E6B3F0E53A
:1007E2000F90E6B4F00209D590E6BAE0FF1212FCCF
:1007F200AA06A9077B01EA49600DEE90E6B3F0EF85
:1008020090E6B4F00209D590E6A0E04401F00209B6
:10081200D590E6A0E04401F00209D51214BC020909
:10082200D51214EF0209D51214E70209D51214AA3F
:100832000209D590E6B8E0247F602B14603C2402C4
:1008420060030208CCA213E433FF25E0FFA215E403
:10085200334F90E740F0E4A3F090E68AF090E68B05
:100862007402F00209D5E490E740F0A3F090E68A22
:10087200F090E68B7402F00209D590E6BCE0547E5B
:10088200FF7E00E0D3948040067C007D0180047CE2
:10089200007D00EC4EFEED4F2436F58274003EF5ED
:1008A20083E493FF3395E0FEEF24A1FFEE34E68F5D
:1008B20082F583E0540190E740F0E4A3F090E68AE9
:1008C200F090E68B7402F00209D590E6A0E04401B4
:1008D200F00209D590E6B8E024FE601D2402600310
:1008E2000209D590E6BAE0B40105C2130209D59017
:1008F200E6A0E04401F00209D590E6BAE070589013
:10090200E6BCE0547EFF7E00E0D3948040067C008B
:100912007D0180047C007D00EC4EFEED4F2436F517
:100922008274003EF583E493FF3395E0FEEF24A149
:10093200FFEE34E68F82F583E054FEF090E6BCE0F1
:100942005480FF131313541FFFE0540F2F90E683BC
:10095200F0E04420F0807C90E6A0E04401F0807357
:1009620090E6B8E024FE60202402706790E6BAE0C8
:10097200B40104D213805C90E6BAE0640260549041
:10098200E6A0E04401F0804B90E6BCE0547EFF7E9E
:1009920000E0D3948040067C007D0180047C007DD1
:1009A20000EC4EFEED4F2436F58274003EF583E4F2
:1009B20093FF3395E0FEEF24A1FFEE34E68F82F53C
:1009C20083E04401F0800C120056500790E6A0E04C
:0A09D2004401F090E6A0E04480F03C
:0109DC0022F8
:0300330002001FA9
:04001F0053D8EF3291
:1012CD0030170990E680E0440AF0800790E680E050
:1012DD004408F07FDC7E0512114890E65D74FFF046
:0F12ED0090E65FF05391EF90E680E054F7F02227
:101148008E4C8F4D90E600E054187012E54D240146
:10115800FFE4354CC313F54CEF13F54D801590E6BD
:1011680000E05418FFBF100BE54D25E0F54DE54CA8
:1011780033F54CE54D154DAE4C7002154C4E6005DF
:061188001214CE80EE22DD
:0212FC00A90740
:1012FE00AE14AF158F828E83A3E064037017AD0119
:10130E0019ED7001228F828E83E07C002FFDEC3E62
:09131E00FEAF0580DF7E007F00B8
:0113270022A3
:1014CE007400F58690FDA57C05A3E582458370F931
:0114DE0022EB
:03004300020D00AB
:03005300020D009B
:100D00000214120002146E000214580002142A0089
:100D10000211CB0002118E000200420002004A00C4
:100D200002005200020CFF00020EFF000215030039
:100D30000215040002150500021506000215070041
:100D40000215080002004A000215090002150A00F7
:100D500002150B0002150C0002150D0002150E0005
:100D600002150F0002004A0002004A0002004A0079
:100D700002151000021511000215120002151300D1
:100D800002151400021515000215160002151700B1
:100D9000021518000215190002151A0002151B0091
:100DA00002151C0002151D0002151E0002151F0071
:080DB0000215200002152100CC
:100F0000120100020000004004230502000001025B
:100F100000010A06000200000040010009022E0044
:100F2000010100C0320904000004FF0000000705B1
:100F30000202000200070504020002000705860203
:100F40000002000705880200020009022E000101CC
:100F500000C0320904000004FF000000070502027F
:100F6000400000070504024000000705860240001B
:100F70000007058802400000040309042203500012
:100F800069006E006E00610063006C006500200067
:100F9000530079007300740065006D007300120344
:100FA000440056004300200031003500300042006C
:020FB00000003F
:060AE500011800011900D8
:10137800759850758920758780758DD9758BD9D2E8
:101388008E438E10D2ACD2BCD2AFC2997E007F0001
:011398002232
:10135400E4FFFE7E50901A87E4F0A3DEFC7E007F5B
:1013640050E4F516F517F51CF51DF51AF51B1213C7
:0313740078FEFF01
:011377002253
:03002300020BE9E4
:100BE900C0E0C0F0C083C082C0D075D000C000C0D2
:0D0BF90001C002C003C004C005C006C00753
:100C0600309923C299C3E51D9517E51C9516501614
:100C16007487251DF582E4341AF583E0F599051DE0
:100C2600E51D7002051C309866C298AF99BFAA06EA
:100C3600751A00751B00C3E51B9450E51A94005005
:100C46001674D9251BF582741A351AF583EFF0054B
:100C56001BE51B7002051ABFAA0AE51B14F51875D9
:100C66002AAA802B74D8251BF582741A351AF583A7
:100C7600E0B52A0AE51B14F51912129D801174D8E5
:0F0C8600251BF582741A351AF583E0252AF52A05
:100C9500D007D006D005D004D003D002D001D000B3
:0B0CA500D0D0D082D083D0F0D0E0325D
:10129D00901ADAE064447027901AE2E0FFB401037B
:1012AD00C20422EF7019D204901AE3E0FFB40104D6
:1012BD00C2048005EF7002D204901AE6E0F53D22DB
:100AEB0060801A0001010105253D0107000400008B
:100AFB0007010000FBF3E7E7E7F7F7FF0009121226
:100B0B00C832123F01010101253D0107000002001F
:100B1B0001050000FBF3F7D7D7F7F7FF090912120E
:100B2B00C8F2363F01010105250101070000000055
:100B3B0001020000FBF3F7E7E7E7F7FF00091212EA
:100B4B00C82D123F01010101052E01070000000213
:100B5B0002030000FBF3F7F7D7D7D7FF09091212EF
:0E0B6B0000C8363F471A80800000FF06E411E4
:1010DE0090E60174CEF090E6F574FFF0901A80E081
:1010EE0090E6F3F0901A81E090E6C3F0901A82E059
:1010FE0090E6C1F0901A83E090E6C2F0901A85E077
:10110E0090E6C0F0901A86E090E6F4F075AF0774A2
:10111E001AF59A7400F59B759DE4E4F59EFF90E632
:10112E007BE090E67CF00FBF80F4000000E490E6D8
:09113E00C4F000000090E6C5F0C9
:011147002285
:100CB0008E4C8F4DE4F527F526F525F524E5BB2070
:100CC000E72F7FF07E497D027C00AB27AA26A9256D
:100CD000A824C31210A77002C322E5272401F52718
:100CE000E43526F526E43525F525E43524F524807C
:0F0CF000CCE54C90E6F0F090E6F1E54DF0D32224
:04132800AD07AC065B
:10132C00E4FFE5BB30E7FB90E6F1E0FFE5BB30E71F
:10133C00FB90E6F0E0FE90E6F2E0FBEEEBFF8D8238
:07134C008C83EEF0A3EFF02B
:011353002277
:0814DF00E5BB30E7FB8FBB22E7
:10148400AC0600000090E6D0ECF000000090E6D13D
:03149400EFF02254
:0B002600E5BB30E7FBEF4404F5BB2214
:10149700AC0600000090E6D0ECF000000090E6D12A
:0314A700EFF02241
:100B790060281AEF000000000000000000000000DB
:100B8900000000000000000000000000000000005C
:100B9900000000000000000000000000C106C100C4
:100BA900C112C18AC18E042400000000C10D0231A6
:100BB9000100022B0040C102C109023B0000C1072C
:100BC900C10BC10FC111C101044100030D4004371C
:0F0BD90000000000C104C10C013D00C110C105A6
:040046005380F722CA
:04004E0043800822C1
:040EFB005380EF220F
:0414FF0043801022F4
:0A1442007B017A1A79ED7F0C7E0021
:0C144C0090D000EFF0AE02AF01021328B8
:10139900E4F53FF54074D92540F582E4341AF58324
:1013A900E4F00540E5407002053F6414453F70E5EF
:0113B9002211
:100DB80090E600E054E74410F01214F775B2FBE433
:100DC800F5B375B4FFF5B5F5B6F5805380FC7F0132
:100DD800FE1211484380035380FD75A01012004E87
:100DE8001214FF90E61074A0F090E611F0000000D5
:100DF80090E61274A2F000000090E61374A0F000D0
:100E0800000090E61474E2F000000090E61574E02B
:100E1800F000000090E6917480F0000000F00000FF
:100E28000090E695F0000000F000000090E604F065
:100E38000000007406F0000000E4F090E680E03066
:100E4800E710753101753200752B00752C40D208FA
:100E5800800E753100753220752B02752C00C20882
:070E680012139943AF0122B0
:1013BA0053A0DF53807F7F017E0012114843A02093
:1013CA007F017E001211484380807F017E00021156
:0113DA0048CA
:1004040030066BE5AA20E06690E690E0FE90E69167
:10041400E07C002400F530EC3EF52FE4F53FF54098
:10042400C3E5409530E53F952F503D74002540F5D8
:100434008274F0353FF583E0752800F529740125B1
:1004440040F58274F0353FF583E0FEE4EE42283057
:100454000B09AF29AE28120CB0920B74022540F59B
:1004640040E4353FF53F80B890E6917480F0200079
:100474000302068DE5AA30E50302068D30106612EC
:100484001442901AEEE030E1367B017A1A79D77F74
:10049400067E0012144C901AD7E0B4EE1DA3E0B40B
:1004A400FF18C200C209C210C202C201D20AC207A6
:1004B400E4F53BF53CC20512004E12144280C330F1
:1004C4000203300A0630021D30011AC200C209C2FA
:1004D40010C202C201D20AC207E4F53BF53CC205D0
:1004E400C20B12004E20090302068D121442E4F5D9
:1004F40027F526F525F524901AEDE0A320E459AF5D
:1005040044AE43AD42AC41AB27AA26A925A824C3D7
:100514001210A75043200140121442E5272401F58C
:1005240027E43526F526E43525F525E43524F52498
:10053400AF44AE43AD42AC41AB27AA26A925F8C3CC
:100544001210A770B2120EFB7FF47E011211481232
:1005540014FFD201C20B809FE5AA30E50302068D89
:10056400C3E53C952CE53B952B400302068D200109
:100574001A300A1790D0007480F0300A32AF32AECD
:10058400311214977F021200268024E4F53FF540CF
:1005940074002540F58274F8353FF58374FFF00547
:1005A40040E5407002053FB400E6E53FB402E1E4F3
:1005B400F527F526F525F524300A65E5BB20E76027
:1005C4007FA07E867D017C00AB27AA26A925A824CE
:1005D400C31210A77033C20A200202C20B90E6F5C0
:1005E40074FFF0E4F53FF54074002540F58274F89B
:1005F400353FF58374FFF00540E5407002053FB4D4
:1006040000E6E53FB402E18017E5272401F527E47D
:100614003526F526E43525F525E43524F52480989A
:1006240030081300000090E6987402F0000000E423
:1006340090E699F08011000000E490E698F0000044
:100644000090E6997440F030071400000090E6042E
:100654007480F00000007406F0000000E4F0053C33
:10066400E53C7002053BB52C20E53BB52B1BE4F5BE
:100674003BF53CC209300204D207D209E58030E3DD
:1006840005120046800312004E201203020761E5A2
:10069400AA30E203020761121442901AEEE030E13C
:1006A400127B017A1A79D77F067E0012144C121439
:1006B4004280E7901AEDE0A320E41E901AEEE030A9
:1006C400E1127B017A1A79D77F067E0012144C124C
:1006D400144280E712144280DA90D0007480F03023
:1006E4000E11E490E695F0AF32AE311214847F011E
:1006F4001214DFE4F527F526F525F524300E3CE544
:10070400BB20E7377FA07E867D017C00AB27AA262D
:10071400A925A824C31210A7400AC20E90E6F574B6
:10072400FFF08017E5272401F527E43526F526E4B4
:100734003525F525E43524F52480C1053CE53C70D8
:1007440002053BB52C17E53BB52B12E58030E405DB
:0E075400120EFB80031214FFE4F53BF53C226D
:02003100D322D8
:02004000D322C9
:0814E70090E6BAE0F53ED322C5
:1014AA0090E740E53EF0E490E68AF090E68B04F09F
:0214BA00D3223B
:0814EF0090E6BAE0F523D322D8
:1014BC0090E740E523F0E490E68AF090E68B04F0A8
:0214CC00D32229
:1000560090E6B9E01210B803E6A402AFA802CEA952
:10006600027DAA01F9AB0221AD024FAE02FBBA0333
:1000760022C400ACC50345CB0088D0009AD100004D
:10008600040090E604E0F54B434B80000000E54B8E
:10009600F002040290E604E0F54B534B7F000000AB
:1000A600E54BF0020402E490E68AF000000090E6D8
:1000B6008BF090E6A0E020E1F990E740E01210B85E
:1000C6000195A600E8A701B3AC01A8B100EEB20104
:1000D60001B30151B40184BC01CDC901DFCD0000DB
:1000E60001F71213BA02040290E741E0B40107D205
:1000F60006D20B020402C20602040290E741E0B4F3
:10010600012A90D0007408F07F017E00120CB0D254
:100116000AD200C20FC21175444075430D754203E1
:10012600754100E4F52FF530D205801790D00074A4
:1001360008F0E4FFFE120CB0D202D210D207D209A8
:1001460012004EE490E6E3F002040290E741E0B4C8
:10015600011390D0007408F07F017E00120CB0D21B
:100166000ED212801190D0007408F0E4FFFE120C3B
:10017600B01214FFC212E490E6DBF002040290E72C
:1001860041E0B40105D209020402C2090204029048
:10019600E741E0B401064380400204025380BF02F7
:1001A600040290E741E090D000F002040290E7419B
:1001B600E0752800F529A3E0FEE4EE4228AF29AE5B
:1001C60028120CB002040290E741E060065380FD5D
:1001D60002040243800202040290E741E0600953F0
:1001E60080DF4380400204024380205380BF020424
:1001F60002D3227E1A7FED121328901AEDE090E7C3
:1002060040F0901AEEE090E741F0E490E68AF000C4
:10021600000090E68B7402F002040290D000740C89
:10022600F07E1A7FED121328901AEDE090E740F069
:10023600901AEEE090E741F0E490E68AF0000000C4
:1002460090E68B7402F002040290D0007406F07EF1
:100256001A7FED121328901AEDE090E740F0901AFD
:10026600EEE090E741F0E490E68AF000000090E6C8
:100276008B7402F0020402E490E68AF0000000901B
:10028600E68BF090E6A0E020E1F990E740E0752DDE
:1002960000F52EA3E0753500F536AF2EFD7AE77B27
:1002A600421213DB9203020402E490E68AF0000095
:1002B6000090E68BF090E6A0E020E1F990E740E0C0
:1002C600753300F534020402AF2EAD347AE77B4075
:1002D6001200035011E490E68AF000000090E68BCD
:1002E600E534F0020402E490E68AF000000090E6AD
:1002F6008BF002040290E680E030E70890E7407455
:1003060001F08005E490E740F0000000E490E68A02
:10031600F000000090E68B04F0020402300B089017
:10032600E7407401F08005E490E740F0000000E447
:1003360090E68AF000000090E68B04F00204027B4F
:10034600017A1A79ED7F267E0012144C901AEDE0A0
:1003560090E740F0901AEEE090E741F07B017A1AC0
:1003660079ED7F247E0012144C901AEDE090E7425E
:10037600F0901AEEE090E743F07B017A1A79ED7F70
:10038600227E0012144C901AEDE090E744F0901A89
:10039600EEE090E745F07B017A1A79ED7F207E004A
:1003A60012144C901AEDE090E746F0901AEEE090A9
:1003B600E747F07B017A1A79ED7F287E0012144C0C
:1003C600901AEDE090E748F0901AEEE090E749F0D9
:1003D600E490E68AF000000090E68B740AF0801C38
:1003E600A205E43390E740F0000000E490E68AF0CE
:0D03F60000000090E68B04F08002D322C3CB
:0104030022D6
:10141200C0E0C083C082D2145391EF90E65D7401A4
:08142200F0D082D083D0E0324B
:10145800C0E0C083C0825391EF90E65D7404F0D081
:0614680082D083D0E032C7
:10146E00C0E0C083C0825391EF90E65D7402F0D06D
:06147E0082D083D0E032B1
:1011CB00C0E0C083C08285100C85110D850D828512
:1011DB000C83A37402F085080E85090F850F828599
:1011EB000E83A37407F05391EF90E65D7410F0D06B
:0611FB0082D083D0E03237
:10142A00C0E0C083C082D2165391EF90E65D740883
:08143A00F0D082D083D0E03233
:10118E00C0E0C083C08290E680E030E72085080C86
:10119E0085090D850D82850C83A37402F085100ED2
:1011AE0085110F850F82850E83A37407F05391EF7F
:0D11BE0090E65D7420F0D082D083D0E03246
:01004200328B
:01004A003283
:01005200327B
:010CFF0032C2
:010EFF0032C0
:0115030032B5
:0115040032B4
:0115050032B3
:0115060032B2
:0115070032B1
:0115080032B0
:0115090032AF
:01150A0032AE
:01150B0032AD
:01150C0032AC
:01150D0032AB
:01150E0032AA
:01150F0032A9
:0115100032A8
:0115110032A7
:0115120032A6
:0115130032A5
:0115140032A4
:0115150032A3
:0115160032A2
:0115170032A1
:0115180032A0
:01151900329F
:01151A00329E
:01151B00329D
:01151C00329C
:01151D00329B
:01151E00329A
:01151F003299
:011520003298
:011521003297
:0814F700E4F54AD2E9D2AF226C
:1012010090E678E020E6F9C2E990E678E04480F0E3
:10121100EF25E090E679F090E678E030E0F990E6AD
:1012210078E04440F090E678E020E6F990E678E056
:0612310030E1D6D2E922F3
:10126B00A90790E678E020E6F9E54A702390E67846
:10127B00E04480F0E925E090E679F08D45AF03A9D5
:10128B00077546018A478948E4F549754A01D32217
:02129B00C3226C
:10123700A90790E678E020E6F9E54A702590E67878
:10124700E04480F0E925E0440190E679F08D45AF70
:1012570003A9077546018A478948E4F549754A0392
:04126700D322C322A9
:03004B000209DDCA
:1009DD00C0E0C083C082C085C084C086758600C05B
:1009ED00D075D000C000C001C002C003C006C00752
:1009FD0090E678E030E206754A06020AC790E6787E
:100A0D00E020E10CE54A64026006754A07020AC758
:100A1D00E54A24FE605F14603624FE7003020AB8B6
:100A2D0024FC7003020AC424086003020AC7AB4603
:100A3D00AA47A948AF4905498F82758300121058FE
:100A4D0090E679F0E54965457070754A05806B90C3
:100A5D00E679E0AB46AA47A948AE498E8275830078
:100A6D00121085754A02E5456401704E90E678E0F6
:100A7D004420F08045E54524FEB5490790E678E031
:100A8D004420F0E54514B5490A90E678E04440F07D
:100A9D00754A0090E679E0AB46AA47A948AE498E63
:100AAD00827583001210850549800F90E678E04429
:100ABD0040F0754A008003754A005391DFD007D08E
:100ACD0006D003D002D001D000D0D0D086D084D0B3
:080ADD0085D082D083D0E03205
:10000300121237E54A24FA600E146006240770F3CF
:0C001300D322E4F54AD322E4F54AD322BC
:1013DB0012126BE54A24FA600E146006240770F3B0
:0C13EB00D322E4F54AD322E4F54AD322D1
:03000000020E6F7E
:0C0E6F00787FE4F6D8FD75814D020EB6C8
:10105800BB010CE58229F582E5833AF583E022504D
:1010680006E92582F8E622BBFE06E92582F8E22297
:0D107800E58229F582E5833AF583E49322B1
:10108500F8BB010DE58229F582E5833AF583E8F0A1
:10109500225006E92582C8F622BBFE05E92582C84D
:0210A500F22235
:1010A700EB9FF5F0EA9E42F0E99D42F0E89C45F09F
:0110B7002216
:1010B800D083D082F8E4937012740193700DA3A3C7
:1010C80093F8740193F5828883E4737402936860DB
:0610D800EFA3A3A380DFDB
:100E7B00020FB2E493A3F8E493A34003F68001F2CC
:100E8B0008DFF48029E493A3F85407240CC8C33378
:100E9B00C4540F4420C8834004F456800146F6DF47
:100EAB00E4800B0102040810204080900AE5E47EE8
:100EBB00019360BCA3FF543F30E509541FFEE4933C
:100ECB00A360010ECF54C025E060A840B8E493A303
:100EDB00FAE493A3F8E493A3C8C582C8CAC583CA2E
:100EEB00F0A3C8C582C8CAC583CADFE9DEE780BEE6
:010BE800000C
:00000001FF
